:02000000F028E6
:100008000800A501A400B9172730A3001030182054
:100018000330A300E8301820A30164301820A3019E
:100028000A30182024082328A2002508A100240843
:10003800A000B9202008031DB913B91B0800303EE1
:10004800A6003C0884000930A70003103020A60C45
:10005800A70B2A28031430288413B91D3F28000849
:100068003A04391D3A068000841700083A04031C34
:100078003A0680004A2800083A04031C3A0639194F
:100088003A06800084173A0980054A28390D06394E
:10009800A0005320A100A00A532000007C280030B3
:1000A8008A0020088207013475340334153400347B
:1000B8003C340C34D934210820040319A00A8030B8
:1000C800201AA1062019A106A018A106210DA00D2D
:1000D800A10DEB28A301A200FF30A207031CA30770
:1000E800031CEB280330A100DF307C207028A1011D
:1000F800E83EA000A109FC30031C8528A0070318CE
:100108008228A0076400A10F822820188B28A01C31
:100118008F2800008F280800A101A301A200023047
:10012800A228A101A301A2000330A228A200013045
:10013800A228A2000430A228A2000530A8002308A3
:100148002102031DA92822082002043003180130C7
:10015800031902302805031DFF30EB280038031D62
:10016800FF300405031DFF30EB28A501A401103062
:10017800A600210DA40DA50D2208A4022308031C26
:10018800230FA5020318CF282208A4072308031861
:10019800230FA5070310A00DA10DA60BBD2820084D
:1001A800EB281030A800A101A001A70CA60C031C85
:1001B800E3282208A00723080318230FA107A10C8E
:1001C800A00CA50CA40CA80BD9282408EB28831391
:1001D80003138312640008008B17F5288B1B080093
:1001E800DE2BF22090308B00F220831681138312CD
:1001F800F22007309F00F2208316713086008312A8
:10020800F220831685018312F2204130C800C9010B
:10021800F2204630D600D701F220D201D301F220D5
:100228003C30D400D501F220F729F22006158316B8
:1002380006118312F2200800F22086148316861015
:100248008312F2200800F220861483168610831287
:10025800F2200615831606118312F2200800F220F8
:100268000611831606118312F2200800F220861068
:10027800831686108312F2200800F2208610831657
:1002880086108312F2200611831606118312F220BB
:100298000800F2208610831686108312F2200611B9
:1002A800831606118312F2200800F2200615831621
:1002B80006118312F2200800F22086148316861095
:1002C8008312F2200800F220861483168610831207
:1002D800F2200615831606118312F2200800F22078
:1002E8000611831606118312F2200800F2208610E8
:1002F800831686108312F2200800F220CA01CB016F
:10030800F2203B30D800640000305802031CEB296F
:10031800F22064005C1CA229F22064005C1D9E2966
:10032800F2203730D800F22014307B20F2205C1104
:10033800F2209F29F220F2205C10F220F2204D21B9
:10034800F22048085602B2004908031C013E570231
:10035800B3000310B30CB20C3308A10032087C20A0
:10036800F22064005D085802031DBD29F2206721B0
:10037800F220F22064005B085802031DC629F2200F
:100388005921F220F220640059085802031DCF2990
:10039800F2206021F220F2204908A10048087C20C0
:1003A800F2204D21F22048085602B2004908031CE9
:1003B800013E5702B3000310B30CB20C3308A1007E
:1003C80032087C20F2200130D80203188729F22055
:1003D8006400DC18F329F2204D21F220EC29F220E8
:1003E800DC10F22081290530BC000430BA00063048
:1003F800B900483024206130242072302420643031
:1004080024202030242044302420723024206930D5
:1004180024207630242065302420203024204330C6
:1004280024206C3024206F302420633024206B304B
:1004380024202030242076302420313024202E30EF
:1004480024203030242008230530BC000430BA00B2
:100458000630B900283024204330242029302420B5
:1004680020302420413024206C3024206130242086
:100478006E30242020302420503024206130242065
:1004880072302420653024206B30242068302420EA
:10049800082320210130A3002C306F203A21192194
:1004A8000130A3002C306F2033210130C200C3017A
:1004B8004208A0004308A1000130A3002C309A2074
:1004C800031DC42A192132307B2033214408A0009F
:1004D8004508A1005F202008C4002108C500440881
:1004E800A0004508A1007030A2001730A300B92071
:1004F8002408B2002508B3003308A10032087C2084
:10050800202132307B203A214408A0004508A10070
:100518005F202008C4002108C5004408A000450841
:10052800A1007030A2001730A300B9202408B2003F
:100538002508B3003308A10032087C202721323077
:100548007B2041214408A0004508A1005F20200825
:10055800C4002108C5004408A0004508A100703067
:10056800A2001730A300B9202408B2002508B30060
:100578003308A10032087C20C20A0319C30F5C2A81
:100588000130C200C3014208A0004308A1000130A5
:10059800A300F4309A20031DED2A1921C8307B20CE
:1005A80033210730A100D0307C202021C8307B20A7
:1005B8003A210730A100D0307C202721C8307B2089
:1005C80041210730A100D0307C20C20A0319C30F93
:1005D800C72AD001D101CE01CF01F5221523F2207F
:1005E8008129F2200230DA00F2202D30DB00F220DF
:1005F800DD01F2205A08A600A7010530A200A301D8
:10060800D520D900F2200800F2200530BC000430C3
:10061800BA000630B9000A3024200D302420F22018
:100628000800F2200530BC000430BA000630B900DA
:100638004D302420203024203A302420203024201B
:100648005B080520F2200823F2200530BC000430A6
:10065800BA000630B90048302420203024203A302F
:100668002420203024205A080520F2200823F220D4
:100678000530BC000430BA000630B90053302420DD
:10068800203024203A302420203024205D08052002
:10069800F2200823F2200530BC000430BA000630EE
:1006A800B900523024206F30242074302420613067
:1006B800242074302420693024206F3024206E30A8
:1006C800242073302420493024206E3024204130E7
:1006D80024205330242065302420633024206F30B8
:1006E80024206E30242064302420633024206F308E
:1006F8002420753024206E30242074302420653066
:10070800242072302420203024203A302420203025
:1007180024205308A50052080620F2200823F220BE
:100728000530BC000430BA000630B900523024202D
:100738006F30242074302420613024207430242029
:10074800693024206F3024206E3024207330242018
:10075800493024206E302420413024205330242076
:1007680065302420633024206F3024206E3024200C
:100778006430242053302420653024207430242011
:10078800503024206F302420693024206E302420FB
:1007980074302420203024203A3024202030242093
:1007A8005508A50054080620F2200823F220082343
:1007B800F2200800DC1486108316861083120611B6
:1007C8008316061183125208A0005308A1001430A2
:1007D800A200A301B9202408B2002508B3003208FA
:1007E800A0003308A100A3010030A020031D2E2C77
:1007F8005C146400061A012CDD016400861A0C2CB6
:1008080064003B305B02031C0B2CDB010C2CDB0A65
:100818006400061B2E2C64000B305A02031C162C95
:10082800DA01172CDA0A5A08A600A7010530A20037
:10083800A301D520B2002508B3005B08A000A101E0
:100848000C30A200A301B920B4002108B500320879
:100858003407D9005208A0005308A1005508A30086
:1008680054089D20031DB12C5C1564003B305D02CB
:10087800031C402CDD01412CDD0A5D08A00000307E
:100888009020B2005B08A0003B309520B4003208ED
:1008980084003408B220B400B5006400340835047C
:1008A8000319582CDB015E2C64005D08003C031D15
:1008B8005E2CDB0A5D08A00000309020B2005B08C7
:1008C800A00000309020B400320884003408B22020
:1008D800B400B5005A08A0000B309520B6003408C3
:1008E800350484003608B220B600B7006400360824
:1008F80037040319812CDA01972C5D08A000003019
:100908009020B2005B08A00000309020B4003208AC
:1009180084003408B220B400B500640034083504FB
:100928000319972CDA0A5A08A600A7010530A20075
:10093800A301D520B2002508B3005B08A000A101DF
:100948000C30A200A301B920B4002108B500320878
:100958003407D900D201D301B42CD20A0319D30A1F
:0A0968008B100900F2206300B72C89
:02400E00553F1C
:00000001FF
